:100000003c373c343c343c37ac0014240c000834fe
:1000100034a33440034003403403a0348010241040
:10002000a0033490001000248c003014009000a035
:100030002490001400030030248c00301424a0030a
:1000400000248c0330900010002400a024900014a1
:10005000002403a0302403a0302403a08f0030101c
:10006000003c3410008f0000af8f030027afafaf0c
:10007000afaf00243c3616020000260c300200020e
:100080000002000016008f8f8f8f8f0327100090c3
:1000900000a02424001424030010009090241024b5
:1000a00010242400140000030027af0c000c008f64
:1000b00000032727afafafaf243cac003c243c2467
:1000c0003c240000ac0000ac008c0010008c000050
:1000d000ac262a14003c243c8c00000024ac0024f4
:1000e0003c243c242600008c000014000000008cfe
:1000f0001000002600008c0000ac00008c00000006
:10010000ac262a14263c24ac3cac3c0c24003c24f9
:100110003c0000900c260c262a14003c0c243c0cbd
:1001200024003c243c0000900c260c262a14003ca1
:100130000c248f8f8f8f032727afafafaf3c243caa
:100140008c00ac24ac24000024243c243c2400007b
:100150002618ac00008c001000008c00022814004f
:100160002400300028102424000024000000008c0b
:100170008c000010ac00002400008c00ac241c009b
:100180008d0000008c00022814002400300028108c
:10019000242400008c00ad262a1400003c243c24ba
:1001a00000008c0000008c00ac262a14003c0c24bb
:1001b000003c243c0000900c260c262a14003c0c29
:1001c000248f8f8f8f03270024002404a0243c2435
:1001d000243c01243c24019090000000008c00107d
:1001e0002400008c00100028140024003000281087
:1001f00024240000009090000010a0009000a02493
:100200001c008d0000281400240030002810242435
:1002100000009010a00090241ca0a0250500030061
:1002200027afaf00243c24000302900000008c2480
:1002300004ac0024243c243c24000100038c001066
:10024000000000022814002400300028102424009c
:10025000008c000125291400000300008c00ac2450
:10026000281400142410002700002404ac2418af24
:100270003c248c0000008c00af2400103c24272478
:100280003c2400008c24192500018c0000008c0007
:10029000110128140024003000281024240001003b
:1002a000008c8c0000ac251d252400140000273c88
:1002b00024270000008c0000008c00ac24281400cf
:1002c00000012529102427273c243c240019000084
:1002d000018c00100100018c001000008c10000047
:1002e00030002810242400008c000024001400009a
:1002f000008c0014002427270000008c2404ac107c
:10030000af8f00af272700018c0010002814242491
:10031000003000281024242400010100008c8c00ef
:100320000010ac240001018c00ac24281400000152
:10033000240014270000270001018c001000008c0d
:100340000000242814002400300028102424100069
:1003500024ac24281400102424270000008c24043a
:10036000acaf24270001008c2404ac252914000024
:1003700001273c242400008c0000008c0010ac00fd
:10038000242814002427270000008c2404ac002417
:1003900027243c2401192400008c0010012814009b
:1003a00024003000281024240000ac00008c000041
:1003b000251d00140003ac0000ac252428140011f6
:1003c000001024032724273c2400011000010525e8
:1003d0000000008c001000008c001000102800307d
:1003e000002810242400008c0001250525110000a0
:1003f000033c2400008c00ac242814242505af27de
:1004000000273c24030400000100018c0010008c34
:1004100000000002281400240030002810242400ca
:10042000008c000024040024240030002810242420
:1004300000018c012814002424000400270001245a
:1004400000018c0010008c00000002281400240021
:1004500030002810242400008c0000240400001028
:100460000010003c24000000008c8c000000008c78
:100470000024002814002400300028102424000345
:100480008c0002000090900000a0250500018f8fd5
:10049000032727afafafafaf000000270000ac24a9
:1004a00028140024270c001600000000028c000213
:1004b0008c00ac261eac1a00270000008c00ac2477
:1004c0000014008f8f8f8f8f032727af0c00301001
:1004d000008f00032727afafafafafafafafafaf66
:1004e00024243c0c243c0c240c243c0c240c243ce4
:1004f0000c240c243c0c243c0c240c023c0c240c3e
:10050000033c0c240c003c0c24af2410af3c2424ee
:1005100000af3c3c24240010003c0c240c023c0c9a
:10052000243c0c24000c0002a0262a14020c263cb9
:10053000240c02008f000010003c0c2412000c263a
:1005400000008c0c260214003c0c24008f000010cc
:10055000243c0c24020202103c020c2600008c0ced
:100560002602143c0c2424100002900c260c262a8f
:1005700014023c0c243c243c240c240210003c2497
:10058000020c0000008c0000900000260214a03c29
:10059000243c240c022410003c0c240c0224163ca5
:1005a0008f0024af3c1024243c240c24103c8f00ea
:1005b00024af240c00262a14243c0c240c243c0ccc
:1005c000248f0c003c0c248f0c003c0c243c0c248d
:1005d000008f8f8f8f8f8f8f8f8f8f03270000005b
:1005e00000000069786d200a41612070477500495c
:1005f000612079726f7420202075690a522d6f2056
:1006000065206f2000297420737365725769206517
:10061000726e657520652020726961696f686f0070
:10062000495f440020614d6e6e65740a6167206ffa
:1006300067652072726365645265656574667500ee
:100640002065746464206c21207273206f67696573
:100650000020206564206f3a24690000000000003b
:10066000000000000000000000000000000000008a
:10067000000000000000000000000000000000007a
:10068000000000000000000000000000000000006a
:10069000000000000000000000000000000000005a
:00000001ff
